:020000040800F2
:10000000000900208D06000851150008551500084C
:100010009115000855150008711500088F06000895
:100020008F0600088F0600088F0600087137000849
:100030008F0600088F0600088F060008FD3B0008A9
:100040008F0600088F0600088F0600088F0600083C
:100050008F0600088F060008DD390008093A0008FD
:10006000353A0008613A00088D3A00088F0600080A
:100070008F0600088F0600088F0600088F0600080C
:100080008F0600088F0600088F060008B1260008BA
:100090002127000881270008E1270008B93A000855
:1000A0008F0600088F0600088F0600088F060008DC
:1000B0008F0600088F0600088F0600088F060008CC
:1000C0008F0600088F0600088F0600088F060008BC
:1000D0008F0600081D2C0008312C00088F06000830
:1000E000213B00088F0600088F0600088F060008D5
:1000F0008F0600088F0600088F0600088F0600088C
:100100008F0600088F0600088F0600088F0600087B
:100110008F0600088F0600088F0600088F0600086B
:100120008F0600088F0600088F0600088F0600085B
:100130008F0600088F0600088F0600088F0600084B
:100140008F0600088F0600088F0600088F0600083B
:100150008F0600088F0600088F0600088F0600082B
:10016000D0400B1CD1409C46203AD3401843524209
:1001700063469340184370479140031C90409C464F
:10018000203A9340194352426346D3401943704783
:1001900080F0004002E000BF81F0004142001FBF3C
:1001A0005FEA410392EA030F7FEA226C7FEA236C45
:1001B0006AD04FEA1262D2EB1363C1BFD21841403A
:1001C00048404140B8BF5B42192B88BF704710F0D0
:1001D000004F40F4000020F07F4018BF404211F073
:1001E000004F41F4000121F07F4118BF494292EADB
:1001F000030F3FD0A2F1010241FA03FC10EB0C0007
:10020000C3F1200301FA03F100F0004302D5494293
:1002100060EB4000B0F5000F13D3B0F1807F06D340
:1002200040084FEA310102F10102FE2A51D2B1F138
:10023000004F40EBC25008BF20F0010040EA03002D
:100240007047490040EB000010F4000FA2F10102DA
:10025000EDD1B0FA80FCACF1080CB2EB0C0200FA64
:100260000CF0AABF00EBC25052421843BCBFD040B2
:100270001843704792F0000F81F4000106BF80F42C
:1002800000000132013BB5E74FEA41037FEA226CEF
:1002900018BF7FEA236C21D092EA030F04D092F0BA
:1002A000000F08BF0846704790EA010F1CBF0020EE
:1002B000704712F07F4F04D1400028BF40F000404B
:1002C000704712F100723CBF00F50000704700F06B
:1002D000004343F0FE4040F4000070477FEA226292
:1002E00016BF08467FEA23630146420206BF5FEA63
:1002F000412390EA010F40F4800070474FF0000363
:1003000004E000BF10F0004348BF40425FEA000C29
:1003100008BF704743F0964301464FF000001CE0D1
:1003200050EA010208BF70474FF000030AE000BF27
:1003300050EA010208BF704711F0004302D5404265
:1003400061EB41015FEA010C02BF844601460020D7
:1003500043F0B64308BFA3F18053A3F50003BCFAF2
:100360008CF2083AA3EBC25310DB01FA02FC63449F
:1003700000FA02FCC2F12002BCF1004F20FA02F2A6
:1003800043EB020008BF20F00100704702F1200299
:1003900001FA02FCC2F1200250EA4C0021FA02F2FA
:1003A00043EB020008BF20EADC7070474FF0FF0CFF
:1003B0001CEAD0521EBF1CEAD15392EA0C0F93EAFA
:1003C0000C0F6FD01A4480EA010C400218BF5FEA9C
:1003D00041211ED04FF0006343EA501043EA51110F
:1003E000A0FB01310CF00040B1F5000F3EBF490009
:1003F00041EAD3715B0040EA010062F17F02FD2A0D
:100400001DD8B3F1004F40EBC25008BF20F00100EF
:10041000704790F0000F0CF0004C08BF49024CEA06
:10042000502040EA51207F3AC2BFD2F1FF0340EA98
:10043000C250704740F400004FF00003013A5DDC09
:1004400012F1190FDCBF00F000407047C2F100024A
:10045000410021FA02F1C2F1200200FA02FC5FEA37
:10046000310040F1000053EA4C0308BF20EADC7081
:10047000704792F0000F00F0004C02BF400010F4F3
:10048000000F013AF9D040EA0C0093F0000F01F0A0
:10049000004C02BF490011F4000F013BF9D041EAC2
:1004A0000C018FE70CEAD15392EA0C0F18BF93EAC4
:1004B0000C0F0AD030F0004C18BF31F0004CD8D1EE
:1004C00080EA010000F00040704790F0000F17BF75
:1004D00090F0004F084691F0000F91F0004F14D0BB
:1004E00092EA0C0F01D142020FD193EA0C0F03D113
:1004F0004B0218BF084608D180EA010000F0004016
:1005000040F0FE4040F40000704740F0FE4040F4F0
:10051000400070474FF0FF0C1CEAD0521EBF1CEA8F
:10052000D15392EA0C0F93EA0C0F69D0A2EB0302AD
:1005300080EA010C49024FEA402037D04FF0805347
:1005400043EA111143EA10130CF000408B4238BF0C
:100550005B0042F17D024FF4000C8B4224BF5B1A1A
:1005600040EA0C00B3EB510F24BFA3EB510340EA68
:100570005C00B3EB910F24BFA3EB910340EA9C0016
:10058000B3EBD10F24BFA3EBD10340EADC001B0186
:1005900018BF5FEA1C1CE0D1FD2A3FF650AF8B422A
:1005A00040EBC25008BF20F0010070470CF0004C37
:1005B0004CEA50207F32C2BFD2F1FF0340EAC25062
:1005C000704740F400004FF00003013A37E792F023
:1005D000000F00F0004C02BF400010F4000F013A81
:1005E000F9D040EA0C0093F0000F01F0004C02BF7C
:1005F000490011F4000F013BF9D041EA0C0195E7E5
:100600000CEAD15392EA0C0F08D142027FF47DAF7D
:1006100093EA0C0F7FF470AF084676E793EA0C0F6D
:1006200004D14B023FF44CAF08466EE730F0004C6B
:1006300018BF31F0004CCAD130F000427FF45CAFFB
:1006400031F000437FF43CAF5FE700BF42000ED2C1
:10065000B2F1FE4F0BD34FF09E03B3EB126209D4FD
:100660004FEA002343F0004323FA02F070474FF0B3
:100670000000704712F1610F01D1420202D14FF028
:10068000FF3070474FF00000704700BF02E000F0FD
:1006900000F8FEE772B6274880F30888264880F302
:1006A000098826484EF60851CEF200010860022063
:1006B00080F31488BFF36F8F03F08AF803F022F9F8
:1006C0004FF055301E491B4A91423CBF41F8040B84
:1006D000FAE71C49184A91423CBF41F8040BFAE77B
:1006E00019491A4A1A4B9A423EBF51F8040B42F874
:1006F000040BF8E700201749174A91423CBF41F824
:10070000040BFAE703F068F803F0FEF8134C144DFD
:10071000AC4203DA54F8041B8847F9E700F03AF8D2
:10072000104C114DAC4203DA54F8041B8847F9E72A
:1007300003F050B80009002000110020000000085C
:1007400000010020000900203047000800110020AF
:100750007811002078110020042600206001000894
:100760006001000860010008600100082DE9F04FF9
:10077000C1F80CD0C3689D46BDE8F08F002383F319
:1007800011882846A047002002F0D4FD02F07AFD2F
:1007900000DFFEE76FF01702364B2DE9F0411A70CB
:1007A000032200245A7001266FF063029C70DC70F3
:1007B0001C715C719C71DC711C725A729E72DC72CD
:1007C00002F08CFF804602F0CDFF0546D0BB2A4BDD
:1007D000984539D03344984537D0284B28F0FF024C
:1007E0009A4234D15FFA88F000F048FA2E4642F27D
:1007F000107400F071FC00F047FA074658B364BB70
:10080000374635B11E4B984503D0002402F0A2FFB5
:100810002746002002F06CFF1A4B9B6813F0400340
:100820001ED00FB100F030F800F078FC00F016FE9A
:1008300000F0BCFE0546ACB900F0C6FC012002F099
:100840007FFDF8E70646D4E706462C46D1E7064684
:100850004FF47A74CDE70446D3E74FF47A74D0E7C7
:100860001C46E1E700F0A2FE401BA042E4D900F0E4
:100870000BF8DDE778110020010007B0000008B098
:10088000263A09B0000C014010B51B4B1B4953F828
:10089000042F013200D110BD8B42F8D1184C194BF6
:1008A00022689A4226D9184B9B6803F1006303F52E
:1008B000C8439A421ED202F02DFF002000F0E8FD4E
:1008C0000220124B187000F017FE114BDA6900225B
:1008D000DA61D96999699A619B6972B60D4B0E4AC2
:1008E000202113601B68226881F311889D4683F3E1
:1008F0000888104710BD00BFFC6300081C64000896
:1009000004640008FF6300087811002084110020AF
:10091000001002400064000808ED00E049F26900A0
:1009200008490B689AB21B0C00FB02330B6044F2BF
:100930005061054A136898B21B0C01FB003010602F
:1009400080B27047101100200C11002010B5044631
:100950000021102200F0ECFD034B03CB206061600E
:100960001868A06010BD00BFE8F7FF1FF0B5BBB06E
:1009700000F01CFE1D4CA368C31AF92B30D906AD3C
:100980002346A06028220021284601F09BFB04F1A9
:100990000E0000F0C5FD0023C6B2591D5F1CDBB27E
:1009A000B3424FEAC10107DA0E3323440822284636
:1009B00001F088FB3B46F0E70123039308230293F1
:1009C0000B4B207B01933023C1F3CF0105910093A2
:1009D000014604A3D3E900230495064801F042F937
:1009E0003BB0F0BD78F6339F93CACD8DC82100206F
:1009F000D5210020A021002070B50D4614461E46CA
:100A000001F0D6F850B9022E0ED1012C0CD112A350
:100A1000D3E90023C5E90023012070BD052C14D0C3
:100A200003D8012C09D0002070BD282C09D0302C0F
:100A3000F9D10BA3D3E90023ECE70BA3D3E90023FF
:100A4000E8E70BA3D3E90023E4E70BA3D3E90023F2
:100A5000E0E700BFAFF30080401DA12026812A0BF4
:100A600078F6339F93CACD8D9E6AC421818A46EE63
:100A700026417272DF25D7B7F017304A39059E56E6
:100A800038B50D460446034620222846002101F0D1
:100A900019FB22792346032A28BF0322284603F89C
:100AA000042F2021022201F00DFB62792346072A40
:100AB00028BF0722284603F8052F2221032201F030
:100AC00001FBA2792346072A28BF0722284603F8FC
:100AD000062F2521032201F0F5FA284604F1080328
:100AE0001022282101F0EEFA382038BD2DE9F04F10
:100AF000FFB01FAE0CAD40F2791280460F46304673
:100B0000002100F015FD48220021284600F010FDCC
:100B100000F04CFD4FF47A72B0FBF2F0554B0DF142
:100B20005209186093E8070001232B74002385E81D
:100B300007000DF152006B74FFF708FF032385F8DF
:100B40002030E82385F8213006AB18464A4903F0E7
:100B5000BFF8172228643146284685F83C20FFF765
:100B60008FFF10AB044601460822304601F0AAFA76
:100B700008220DF14103A118304601F0A3FA0DF14E
:100B80004203082204F11001304601F09BFA11AB38
:100B9000202204F11801304601F094FA12AB4022F1
:100BA00004F13801304601F08DFA14AB082204F14B
:100BB0007801304601F086FA0DF15103082204F164
:100BC0008001304601F07EFA04F1880A04F5847B46
:100BD0004B465146082230460AF1080A01F072FAE3
:100BE000D34509F10109F3D119AB08225946304622
:100BF00001F068FA4FF0000904F5887495F8343074
:100C00004B4510D84FF0000995F83C304B4515D9AD
:100C10002B6C21464B440822304601F053FA08342D
:100C200009F10109F0E7AB6B21464B44082230463D
:100C300001F048FA083409F10109DFE7E31DC3F3C5
:100C4000CF03F97E0593002304960393BB7E1937E7
:100C50000293012301970093404604A3D3E90023A4
:100C600001F000F87FB0BDE8F08F00BF9E6AC4219C
:100C7000818A46EE88110020883E0008014B1870DA
:100C8000704700BF94110020F0B5264B85B01C7B47
:100C900084B9254A02AB1068516803C3082323496D
:100CA0000DEB0302224802F0F5FF054620B921486A
:100CB00000F046FC002032E00369B3F5CE3F04D9D2
:100CC00019461D4800F03CFCF4E7418BB1F57A7FF2
:100CD00005D04FF47A72194800F032FCEAE7184A5E
:100CE000103B0244124920469E1A00F063FC07465E
:100CF00005F118013246204600F05CFCA9688F42DD
:100D000002D1EB68984206D000903B46EA680D4855
:100D100000F016FCCEE70C4800F012FC012005B0F4
:100D2000F0BD00BFC8210020783D0008DC9B010019
:100D300000640008803D00088C3D00089E3D0008CE
:100D4000089CFFF7BC3D0008E53D00082DE9F04F89
:100D5000AFB006AF80460D4600F02AFF04460028DB
:100D60006FD12B7E022B1BD1EB8A012B18D100F007
:100D70001DFC8146FFF7D2FDFFF7C0FAA749FFF738
:100D8000C9FBA749FFF712FBFFF760FCA54E09F569
:100D90001679EB7E4844306093B90022A24B1A705A
:100DA000A437BD46BDE8F08F07F10C031C44009446
:100DB000002308224FEAC901284600F0E7FF4C460D
:100DC000AB8A5FFA84F9013BA3420BD904F1010914
:100DD000B9F1110FE8D14FF49871944B944A9548AA
:100DE00002F02AFF07F11C00FFF7B0FD224607F1D1
:100DF0001C0107F10C0002F03DFF03460028CCD196
:100E0000B9F1100F07D0884B83F800903368A3F531
:100E100016733360C4E707F1A00202F8950D01468E
:100E200000922846072200F0B1FFF97A7F2904DDFD
:100E3000814B7F4A40F24711D1E7404600F09CFECB
:100E4000AEE7EB8A052B00F0318106D8012BA7D144
:100E500029464046FFF74AFEA2E7282B3DD0302B1B
:100E60009ED16B7E754C0133627BDBB29342EA46C6
:100E700040F01A81EA7E237B9A4240F015810026D9
:100E800007F1A00323F8846D00931022012331465B
:100E9000284600F07BFFB5F81480A8F102081FFA7D
:100EA00088F808F1030323F003030A3323F0070350
:100EB000ADEB030D0DF1180933469BB2B11C9845FB
:100EC0004FEAC10106F101066DDD4B440093082293
:100ED0000023284600F05AFFEEE7AB8A013B9BB2A5
:100EE000C92B3FF65DAF554E347B4CBB06F10C036E
:100EF0000093082223462146284600F047FFAB8A8C
:100F000004F10109013BE4B29C424FEAC90109DA4C
:100F10000E343444009400230822284600F036FFA3
:100F20004C46ECE700230022C6E900230023B3600F
:100F300086F8D730C6F8D830337B0BB9EB7E3373E5
:100F4000002407F11C0607F10C0308222146304655
:100F5000FC603C617C6101F0B5F83B7C04F1010967
:100F6000A3424FEAC90107D97B69082223443046CE
:100F700001F0A8F84C46F0E70023C1F3CF01E87E6A
:100F8000059104960393AB7E1935029328230146FD
:100F9000009301951FA3D3E90023404600F062FEB1
:100FA000FFF7E4FCFCE694F8D70000F083FAD4F8ED
:100FB000D83006461BB994F8D70000F08BFAD4F865
:100FC000D83043449E4204D294F8D700013000F058
:100FD00081FA00251A4B4FEA980BAAB25A451046DF
:100FE00030DA5AB994F8D72042B9D4E900120A434A
:100FF00004D1D9F800201A600135EEE7226859F8CB
:10100000201002EB80007B6000F044FA7B68F3E77D
:10101000AFF3008026417272DF25D7B700FF7F470C
:101020000000C8439C21002099210020F43D0008C5
:10103000A03E00084D3E00086F3E0008C821002079
:1010400000110020D4E90023D4F8D85012EB080096
:1010500043F10001C4E90001454494F8D700C4F805
:10106000D85000F027FA854209D394F8D7300133DD
:1010700084F8D730D4F8D8309E1BC4F8D860B8F1C3
:10108000FF0F0ADC0020104B2073196800F002FAF1
:10109000FFF7FAFD08B1FFF7F7FB23680B4A9B0A3D
:1010A000013313810023A360D54679E6BFF34F8F48
:1010B0000749084BCA6802F4E0621343CB60BFF3F0
:1010C0004F8F00BFFDE700BF0011002088110020F6
:1010D00000ED00E00400FA0508B54FF000530B4A9C
:1010E000196891420AD1597D094A0A4811701B7D3D
:1010F000C922037308490E3000F008FABDE8084021
:10110000E02200214FF0005000F012BA9AAD44C521
:1011100094110020C8210020160000201FB50222D3
:101120001D4B00245A710423ADF808300123072217
:101130001A49ADF80C408DF80B308DF80C30184B77
:1011400018484B608DF80A2001F0D8FD164B17495E
:1011500000930194164B4FF48052164800F0D6FCD1
:10116000154B197811B1134800F006FD00F01EFA76
:101170000446FFF7D3FBFFF7C1F81049FFF7CAF9A0
:101180000F49FFF713F9FFF761FA04F516740D4BD9
:1011900004441C6004B010BD88110020041100201C
:1011A00003000600B8220020F90900089811002069
:1011B0004D0D0008A02100209411002000FF7F4762
:1011C0000000C8439C2100202DE9F04F99A7D7E9E2
:1011D00000670FF26829D9E900898F4C93B0DFF8D6
:1011E00064B2DFF864A2204600F088FD0CAD0790E1
:1011F00098B310220021284600F09AF94FF000021F
:10120000079B197B61F3030219468DF8302051F8D2
:10121000040F0EAA496803C21B680D9A584663F36F
:101220001C029DF830300D9243F020038DF83030D1
:1012300000232A46194601F071FD079030B9204677
:1012400000F060FD079B8AF80030CCE79AF8003088
:10125000072B40DC01338AF8003018220021284691
:1012600000F066F9DFF8DCB1DFF8E0A100232A46E0
:101270001946584601F07AFD014680BB102208A8A5
:1012800000F056F9DAF80C3083F01003CAF80C308D
:1012900000F08EF90DF1240E0B4612A9024611E959
:1012A00003008EE803009DF83410C1F303008906A3
:1012B00049BF0E99BDF83810C1F31C0141F000413F
:1012C00058BFC1F30A018DF82C000891204608A9E7
:1012D00000F05EFFCAE7204600F014FDBDE720469F
:1012E00000F066FC834600284BD100F05FF94B4BC1
:1012F0001A68904245D3079300F058F98246FFF7E9
:101300000DFBFEF7FBFF4649FFF704F94549FFF7E0
:101310004DF8FFF79BF98DF820B0DFF834B10AF5EE
:10132000167A079B9BF800105044186011B90123EE
:101330008DF8203028460791FFF708FB07990DF13B
:101340002100C1F1100A5FFA8AFABAF1060F28BF2C
:101350004FF0060A2944524600F0D8F80AF101037A
:10136000049308AB0393182302932F4B3246019347
:101370000123204600933B4600F01CFC00238BF821
:10138000003000F013F9294ADFF8C8A01368C31A27
:10139000B3F57A7F32D3106000F00AF902460B46AB
:1013A000204600F0B5FC204600F002FC30B39AF86D
:1013B0000C30DFF8A4B0002B14BF032302238BF8FA
:1013C000053000F0F3F84FF47A73B0FBF3F02946E0
:1013D000CBF800005846FFF753FB18230293144B39
:1013E0000730019340F25513C0F3CF0004900093EF
:1013F000039542464B46204600F0DCFB9AF80C3041
:101400000BB1FFF7B3FA9AF80C30002B7FF4E7AE7C
:1014100013B0BDE8F08F00BFA02100209C21002068
:1014200000FF7F470000C84398210020A822002029
:10143000AC220020401DA12026812A0BF1C6A7C1A5
:10144000D068080FB8220020AD220020000801401B
:1014500099210020C82100208811002070B502F0D9
:1014600025F80025084C094E207030682378834207
:1014700008D902F017F8336805440133B5F5C84FB1
:101480003360F2D370BD00BFB4220020B022002030
:1014900002F09AB807B502AB43F8041D00F10060F2
:1014A0000422194600F5C84002F03AF803B05DF88E
:1014B00004FB0000054B1A68054B1B789B1A8342FE
:1014C00002D9104401F0EEBF00207047B022002086
:1014D000B422002038B50446064D2868204401F0A7
:1014E000E7FF28B928682044BDE8384001F0F2BF82
:1014F00038BD00BFB0220020022802BF4FF4801286
:10150000014B1A61704700BF00080140002310B56D
:10151000934203D0CC5CC4540133F9E710BD000002
:1015200002460346981A13F9011B0029FAD17047A5
:1015300003460244934202D003F8011BFAE77047C6
:101540000FB4002004B070470EB4002003B0704701
:10155000FEE70000EFF30983EFF30583034B9A6B7B
:101560009A6A9A6A9A6A9A6A9B6AFEE700ED00E0B4
:10157000EFF30983EFF30583044B9A6B9A6A9A6A37
:101580009A6A9A6A9A6A9B6AFEE700BF00ED00E0D9
:10159000EFF30983EFF30583034B5A6B9A6A9A6A58
:1015A0009A6A9A6A9B6AFEE700ED00E002F05AB878
:1015B00002F044B810B5074C0A44914208D011F823
:1015C000013B4340DBB254F8233083EA1020F4E7B8
:1015D00010BD00BFE43E00080246006848B1036841
:1015E00011891360D38801339BB29942D38038BFED
:1015F0001381704770B504460D4688B02022002143
:101600006846FFF795FF20460495FFF7E5FF05467E
:1016100058B16B46044608AE1A4603CAB24220606F
:101620006160134604F10804F6D1284608B070BD85
:101630002DE9F04130B940F2C531264B264A274802
:1016400002F0FAFA0B7C23B9254B234A40F2C6314B
:10165000F5E7C66986B9C161BDE8F081002B29DADA
:10166000930CAB4229D1B44201D10C60F3E7C8F826
:1016700000100C60BDE8F0814B68B04623F0604775
:10168000BD0C15EA230538BF3D4634464FEAD37EEC
:10169000C3F3807C6368BEEBD37F23F06042DDD16F
:1016A000974203D1C3F380739C450AD1974205E06A
:1016B0001C46EFE7AA4206D013469D422CBF0023EA
:1016C0000123002BCFD12368A046002BF0D121604D
:1016D000BDE8F08174450008684300082C46000806
:1016E0004D46000808B5034A034B40F25E310348FB
:1016F00002F0A2FA44430008EC4500082C4600081A
:1017000008B503680B60C388016033B9044B054A10
:101710004FF4C761044802F08FFA013BC38008BD53
:10172000BC450008B84300082C46000870B50C46BC
:1017300000F10C05616831B9E38A002061F3090307
:10174000E382002170BD0E682846FFF7D9FF66606E
:10175000F0E7000008B5426832B10B4B0B4A40F28B
:101760002F410B4802F068FAC37DC3F384010131B5
:1017700061F38603C375C38A62F30903C3821B0A3C
:1017800062F3C713C37508BD084600087443000818
:101790002C4600082DE9F047089E32B91F4B204A1D
:1017A00040F239511F4802F047FA4FF47F4901F0E7
:1017B00007054FEAD6082A4406F0070600EBD100D9
:1017C000954201D1BDE8F08705F0070E06F0070A43
:1017D000D645774638BF5746511BC7F108078F4299
:1017E00028BF0F46EC08045D08EBD60113F801C0D2
:1017F00004FA0EF429FA07FE24FA0AF45FFA8EFEC0
:101800008CEA04044EFA0AFE04EA0E048CEA040C84
:1018100003F801C03D443E44D2E700BF88450008BC
:101820008C4300082C4600082DE9F04106460F467F
:1018300000254FF6FF7441F221082A46304639460A
:10184000FEF78EFC0823C0B284EA002414F4004F93
:101850004FEA4404A4B203F1FF3318BF84EA08043A
:1018600013F0FF03F2D10835402DE6D12046BDE844
:10187000F081000010B541F221040A44914200D1E8
:1018800010BD11F8013B80EA0320082310F4004F3B
:101890004FEA400080B203F1FF3318BF604013F0FD
:1018A000FF03F3D1EAE700002DE9F04F85B08A4647
:1018B0008DE80C00BDF83C40814630B940F26E31F5
:1018C000484B494A494802F0B7F911F0604F04D03B
:1018D000474B454A40F26F31F4E7009B002B7ED026
:1018E00024B10E9B002B7AD0072C28D809F10C00CC
:1018F000FFF772FE054628B96FF00205284605B0CD
:10190000BDE8F08F14220021FFF712FE22460E9947
:1019100005F10800FFF7FAFD631C2B74009B2C44B3
:101920001B78294603F01F0363F03F0323724AF03C
:1019300000436B604846FFF77BFE0125DEE74FF072
:1019400000084FF0800B46464546019B1B0A029358
:1019500000F10C0303930398FFF73EFE07460028AF
:10196000CAD014220021FFF7E3FDB6BB02229DF886
:1019700004303B729DF808307B720E9B711E194437
:10198000B4420AD9B818013211F801EFD2B20136C7
:10199000072A80F808E0B6B2F2D1B44208BF4FF08F
:1019A000400B009BB8181978013201F01F0141EA81
:1019B00048114BEA010303724AF000437B603A741A
:1019C00039464846FFF734FE0135B4422DB288F05F
:1019D00001084FF0000BBED190E70022CDE76FF079
:1019E00001058BE774450008584300082C460008A1
:1019F000984500082DE9F0471E46CB8A9146C3F36F
:101A00000902062A80460F4619D013460021B0B2BB
:101A10008DB25A1992B2052A09D9A84210D8FA8A69
:101A2000034463F30902FA820120BDE8F087A8426B
:101A3000F3D919F801403A4494760131E8E70025DA
:101A4000FB8A7C68C3F309001C23821FB2FBF3FAF4
:101A500003FB1A2A1FFA8AF27CB301212368002BA8
:101A600039D1B31F03441C20B3FBF0F301339BB205
:101A700099420CD2BAF1000F09D14046FFF7ACFDF4
:101A800008B1C0F800A0206008B3044600224FF05F
:101A9000000AB6B2B54230D21346691E4944E01876
:101AA000013311F801EF9BB201351C2B80F804E0E3
:101AB000ADB214D0AE42F2D8ECE74046FFF78CFD51
:101AC000044608B1002303607C60002CDED16FF077
:101AD0000200BDE8F087013189B21C46BEE7AE4284
:101AE000D8D94046FFF778FD08B1C0F800A02060C3
:101AF0000028ECD004460022CCE7FB8AC3F309029D
:101B0000164466F30903FB828EE70000F8B50E4623
:101B100015461F46044628B9144B154A4F2115484F
:101B200002F08AF824220021FFF702FD069B6A09D1
:101B30006360079B002023624FF6FF739A4228BF21
:101B40001A46A7602070A061E06197B204F10C050D
:101B5000824205D100232B6027826382A382F8BDD5
:101B60002E60013035462036F2E700BF7045000890
:101B7000E44200082C46000808B528B97321084B38
:101B8000084A094802F058F8037823B94BB2002BF1
:101B900001DD017008BD054B024A7D21F1E700BF60
:101BA00074450008F04200082C460008B8440008BC
:101BB000007870472DE9F7430D9E074619461046F9
:101BC000BDF828900B9D9DF83040BDF8388016B9BF
:101BD000B8F1000F43D11F2C41D83B78D3B9B8F1ED
:101BE000070F39D839F0030339D1424631464FF651
:101BF000FF70FFF73FFE4FEA092920F0010009F4CA
:101C00004079400449EA0464400C44EA40244FF619
:101C1000FF730DE043EA0923B8F1070F43EA0464B8
:101C2000F5D9FFF701FE42463146FFF723FE034692
:101C30008DE840012A4621463846FFF735FE0DB9AA
:101C4000FFF750FD2B780133DBB21F2B88BF002339
:101C50002B7003B0BDE8F0836FF00300F9E76FF07D
:101C60000100F6E72DE9F7430E9F81460B9D9DF895
:101C700030009DF83480BDF83C6007B9C6BB1F2812
:101C800036D899F800E0BEF1000F34D00C0244F0D1
:101C900080049DF8281044EAC83444EA014444EA28
:101CA0000E04072E44EA006415D919461046FFF7C2
:101CB000BBFD32463946FFF7DDFD0346019600972E
:101CC0002A4621464846FFF7EFFDB8F1010F0CD137
:101CD00025B9FFF707FD4FF6FF73EFE72B780133C8
:101CE000DBB21F2B88BF00232B7003B0BDE8F0834D
:101CF0006FF00100F9E76FF00300F6E7C06900B18B
:101D000004307047C1690C300B680361FFF7F8BC01
:101D10002DE9F84FD0F818A0054616461F46544640
:101D20004FF00009DFF8608000F10C0B0CB9BDE842
:101D3000F88FD4E90223B21A67EB0303994508BF71
:101D400090451FD2AB6921469C4228460DD1FFF732
:101D5000EDFCAB6921461B685846AB61FFF7D0FC30
:101D6000AC692346A2461C46E0E7FFF7DFFC236888
:101D70002146CAF800305846FFF7C2FC5446DAF84C
:101D80000030EFE72368EDE780841E002DE9F04F77
:101D90008BB00D4614460793DDF85090824600281C
:101DA00000F06481B9F1000F00F06081531E3F2BF9
:101DB00000F25C81012A03D1079B002B40F0568181
:101DC0000023BAF814600893F600B542099380F036
:101DD00053812B199E420AD2761B16F0FF0607D1BB
:101DE00040F26751AA4BAB4AAB4801F025FF2646AB
:101DF000DAF80C3023B9DAF81030002B00F0A580A7
:101E00002F2D31D8C5F1300846454FF0000334BFBF
:101E1000B0465FFA88F80093294608AB4246DAF8E4
:101E20000800FFF7B7FCA6EB08074544FFB24FF0E8
:101E3000300BBAF8143003F10053063BDB00029379
:101E4000DAF80C300593059B002B51D087B9DAF8EE
:101E50001000002861D0002F5FD0AB4550D98F4BC8
:101E60008C4A40F2A651BFE737464FF00008DEE744
:101E7000029B23B98A4B874A4FF4B161B4E7029BB6
:101E8000E02B28BFE02306935B44AB4204931DD9AB
:101E90005B1B9F4226BFDBB203930397AB4504D97C
:101EA0007E4B7C4A40F291519EE70598CDF8008028
:101EB00008ABA5EB0B01039A0430FFF76BFC039B07
:101EC0009844FF1A1D445FFA88F8FFB2049B9B45B3
:101ED00004D3744B6F4A40F29B5185E7029B069AEC
:101EE000DDF810B09B1A0293059B1B680593AAE7C7
:101EF000029BBB42ABD26C4B664A40F2A15173E7E6
:101F0000CDF800803A46A5EB0B0108ABB8443D4440
:101F1000FFF740FC00275FFA88F8BAF81430B5EBF9
:101F2000C30F04D9614B5B4A40F2B1515CE7B8F191
:101F3000400F04D95E4B574A40F2B25154E767B1A3
:101F40005C4B544A40F2B3514EE70093324608AB23
:101F50002946DAF80800FFF71DFC731E3F2B35B247
:101F600001D8A64204DD544B544A40F235213BE7E8
:101F700060070AD00AAB03EBD40111F8083C6242B7
:101F800002F00702134101F8083C082C21D9102C5B
:101F900021D9202C8CBF08230423079A002A6DD056
:101FA000B4EBC30F6CD0082C04F1FF3215D89DF8A8
:101FB000203023FA02F2D10706D54FF0FF3202FAA1
:101FC00004F423438DF820309DF8203089F8003048
:101FD0004EE00123E1E70223DFE7102C11D8BDF822
:101FE000203023FA02F2D20706D54FF0FF3202FA70
:101FF00004F42343ADF82030BDF82030A9F80030B8
:1020000036E0202C0ED8089921FA02F2D30705D524
:102010004FF0FF3303FA04F40C430894089BC9F80B
:10202000003025E0402C1CD0DDE9086730463946F9
:10203000FEF796F8002100F0010050EA01030BD0F2
:10204000224601200021FEF797F8404261EB410152
:1020500006430F43CDE90867DDE90823C9E90023FA
:1020600006E0174B154A4FF42071BDE66FF00105ED
:1020700028460BB0BDE8F08F1D46F9E7012CA3D030
:10208000082CA1D9102CB7D9202CE5D8C6E700BF61
:10209000C44300089C4300082C460008E64300089F
:1020A000D34300080B440008334400085A44000896
:1020B00088440008A0440008BA4400081C430008F3
:1020C000B844000830B585B030B940F2B121234B97
:1020D000234A244801F0B0FD23B9234B204A40F2A3
:1020E000B221F6E7402A04D9204B1D4A40F2B6211E
:1020F000EFE722B91D4B1A4A4FF42F71E9E700248C
:10210000012A0294039417D11B788DF808305307E5
:102110000AD004AB03EBD20313F8084C554205F088
:102120000705AC4003F8084C00910346002102A8C3
:10213000FFF730FB05B030BD082AE5D9102A03D8D7
:102140001B88ADF80830E2E7202A02D81B6802930A
:10215000DDE7D3E90045CDE90245D8E7F4440008BE
:10216000304300082C4600080F450008B84400081A
:1021700070B50C4600F10C05E16819B9A160216148
:10218000A18270BD0E682846FFF7BAFAE660F3E751
:102190002DE9F04FD1F8009091B0C9F3C016044674
:1021A0000D46CDE90223002E50D0C9F3C03BC9F340
:1021B0000626B9F1000F80F29F8119F0C04F40F060
:1021C0009B812B7B002B00F09781BBF1020F03D08A
:1021D0002278B24240F0938109F07F02BBF1020FF6
:1021E000059236D119F07F0FC9F30F2A01D10AF0F9
:1021F000030A2B447606059A93F8038046EA0B46B9
:1022000046EA82465FEAD81346EA0A06069300F0D9
:102210009A800022002310A961E90823059B6768C2
:10222000009352465B462046B847002800F088805D
:10223000A7698FB9314604F10C00FFF7DBF90746B7
:10224000D0B96FF0020011B0BDE8F08F4FF0020B73
:10225000AFE7C9F3074ACCE73B699E420DD03F6820
:10226000002FF9D1314604F10C00FFF7C3F90746FE
:102270000028E6D0A3693B60A761DDE90801FFF70C
:10228000D3FAB882F97D08F01F06C1F38401711AF0
:1022900089B20FFA81FEBEF1000FB8BF01F1200E26
:1022A000C9F30461D7E90223B8BF0FFA8EFE079184
:1022B00052EA030100F02F81DDE90201801A61EB8F
:1022C00003010B46002102469E48994208BF9042F6
:1022D000C0F02181069B002B3FD0BEF1010F00F31F
:1022E0001A8118F0400F38D0DDE90223C7E9022334
:1022F000202200210DEB0200FFF71AF9DDE902238D
:10230000CDE908232B1D0A932B7B2046013BDBB232
:10231000ADF834309DF81C30ADF836A08DF83A3069
:102320009DF814308DF838B08DF83B308DF8396059
:10233000A36808A998473846FFF70CFA002082E7FF
:102340006FF00B007FE7A76917B96FF00C007AE711
:102350003B699E4296D03F68F6E7FB7DC8F340128A
:10236000B2EBD31F40F0CE80C3F38403B34240F0FE
:10237000CC8006992B7B4FEA981279B3D2073CD4D4
:10238000032B40F2C580DDE90223C7E902232B7B42
:10239000AE1D033BDBB23246394604F10C00FFF7B9
:1023A00029FB002808DA39462046FFF7BFF93846EE
:1023B000FFF7D0F9032046E7AB883B832A7B033A3B
:1023C000D2B2B88A3146FFF755FAFB7DB882DA43BC
:1023D000C2F3C01262F3C713FB75AFE76AB92E1DD3
:1023E000013BDBB23246394604F10C00FFF702FB39
:1023F0000028D8DB2A7B013AE2E7FA8A013BC2F3E4
:102400000902052AD9B250D80023281D99420AD9B9
:1024100007EB020E10F801CB01320133062A8EF8C9
:102420001AC0DBB2F2D18B4228BF0023DDE902895A
:1024300007F11A02CDE908890A927A683CBF043391
:102440005B190B920C93FB8AADF836A0C3F309031A
:1024500019449DF81C30ADF834108DF83A309DF8D1
:1024600014308DF838B08DF83B3000238DF839608A
:102470007B602A7BB88A013A291DFFF7FBF93B8B69
:10248000B882834203D1A36808A92046984708A9C7
:102490002046FFF76DFE3846FFF75CF9B88A3B8BA4
:1024A000984214BF11200020CDE6786810B34FF099
:1024B000060E03689BB9A2EB0E021B2A13D8033247
:1024C000024405F1040E1F309942ACD91EF801CB2D
:1024D000013302F801CF9042DBB2F5D1A3E70EF150
:1024E0001C0E1846E5E7184B184A40F2B31118487D
:1024F00001F0A2FB034696E76FF00900A3E66FF038
:102500000A00A0E66FF00D009DE66FF00E009AE65F
:102510006FF00F0097E6FB7D394668F386036FF393
:10252000C713FB752046FFF701F9069B002B7FF4CC
:10253000D8AEFB7DC3F38402013262F38603FB75E0
:1025400003E700BF80841E002445000808430008FC
:102550002C460008026843681143016003B1184724
:10256000704700002DE9F0414E4EB04240F08680A9
:102570004D4CDFF838E1E56945F00075E561E46947
:10258000446DD4F8007207EA0E0747F00107C4F85B
:102590000072D4F8005205EA0E0545F0010545EA3F
:1025A0000121C4F80012002A6AD000210F46C4F8A5
:1025B0001C12C4F80412C4F80C12C4F8141204EB70
:1025C000C10501310E29C5F84072C5F84472F6D133
:1025D0004FF0000E4FF0010C964510D1426DB04205
:1025E000D2F8003223F00103C2F8003258D12E4B4A
:1025F000DA6922F00072DA61DB69BDE8F0819F7868
:102600001D8817F0010F18BFD4F804820CFA05F1E9
:102610001CBF41EA0808C4F8048217F0020F18BF73
:10262000D4F80C8204EBC5051CBF41EA0808C4F8C5
:102630000C827F0748BFD4F8147203F10C0344BF27
:102640000F43C4F8147253F8087C0EF1010EC5F85C
:10265000407253F8047CC5F84472D4F81C522943E4
:10266000C4F81C12B8E70021446DC4F81C12C4F869
:102670000412C4F80C12C4F81412A9E7002AF2D10B
:102680000022436DC3F84022C3F84422C3F8042259
:10269000C3F814220122C3F80C22C3F81C229DE7C0
:1026A000BDE8F081B8220020001002400000FFFFCA
:1026B000184B10B55A6D936813F00104936005D060
:1026C00013F00C0F14BF4FF480340124D90506D544
:1026D00013F4406F14BF44F4003444F00204DA03EE
:1026E00006D513F4402F14BF44F4802444F00404AE
:1026F000202383F311880021074800F049FE21467A
:102700000648FFF727FF002383F31188BDE8104038
:1027100001F038B8B8220020C0220020DC220020BE
:1027200038B5154C636DDD68AA0713D05A6922F0DD
:1027300002025A61202383F31188002104F1100062
:1027400000F026FE012104F11800FFF703FF00232B
:1027500083F31188EB060BD51021636DD96020231C
:1027600083F311880548FFF7F5FE002383F31188F2
:10277000BDE8384001F006B8B8220020E822002069
:1027800038B5154C636D1D69AA0713D05A6922F03C
:1027900010025A61202383F31188002104F11000F4
:1027A00000F0F6FD022104F11800FFF7D3FE00232C
:1027B00083F31188EB060BD51021636D196120237B
:1027C00083F311880548FFF7C5FE002383F31188C2
:1027D000BDE8384000F0D6BFB8220020E822002033
:1027E00038B5144C636D5D682A075D6010D52046CE
:1027F000032200F8482B1A6822F002021A602023F4
:1028000083F311880021FFF7A5FE002383F31188CD
:102810006B070BD5636D9969202383F311880648F4
:102820000904FFF797FE002383F31188BDE83840C1
:1028300000F0A8BFB8220020E822002010B50F4CFD
:10284000204600F03FFA0E4B0B211320636500F089
:1028500019FA0B21142000F015FA0B21152000F0B5
:1028600011FA0B21162000F00DFA00232046BDE8D6
:1028700010401A460E21FFF775BE00BFB822002097
:10288000006400400F4B10B59842044605D10E4B32
:10289000DA6942F00072DA61DB690122636D1A6065
:1028A000636D5A68D20707D5626851681268D961AA
:1028B0001A60064A5A6110BD0121082000F09CFCF4
:1028C000EEE700BFB8220020001002405B87010045
:1028D00003291AD8DFE801F0020A0F14436D9B6840
:1028E00013F0E05F14BF012000207047436D98682B
:1028F000C0F380607047436D9868C0F3C060704754
:10290000436D9868C0F30070704700207047000066
:1029100010B503291FD8DFE801F0021F2327416DFE
:102920008B68C3F30163183301EB0313107881063E
:102930001ED55468C0F30011490041EAC40141F0BA
:10294000040100F00F005860906841F001019860A8
:10295000D268DA60196010BD436D03F5C073E5E716
:10296000436D03F5C873E1E7436D03F5D073DDE70D
:102970009488C0F30011490041EA4451E1E70000A6
:1029800001290CD003D3022910D000207047436DD9
:10299000DA68920701D1186903E001207047436D9E
:1029A000D86810F0030018BF01207047436DF2E7AC
:1029B00010B539B9436DD96889071BD11B699B07CD
:1029C00004D110BD012915D0022948D1416DD1F89B
:1029D000C031D1F8C401D1F8C8411461D1F8CC415B
:1029E000546120240C610C69A40717D14C6944F090
:1029F000100412E0416DD1F8B031D1F8B401D1F832
:102A0000B8411461D1F8BC4154612024CC60CC6839
:102A1000A40703D14C6944F002044C6111795C08AD
:102A200064F304119C0864F34511117189064BBFCE
:102A300091681189DB085B0D4CBF63F31C0163F3E4
:102A40000A01137948BF916060F3030313714FEAE1
:102A500010234FEA104058BF11811370508010BDF1
:102A600000231A4610B51C495A50CC180833802B45
:102A70006260F9D1194B9A6942F07D029A619B69B3
:102A80000268174BDA6082685A6042681A60C2684E
:102A900003F58063DA6042695A6002691A608269EC
:102AA000C3F80C24026AC3F80424C269C3F80024E2
:102AB000426AC3F80C28C26AC3F80428826AC3F8C1
:102AC0000028026BC3F80C2C826BC3F8042C426BF9
:102AD000C3F8002C10BD00BF1023002000100240DE
:102AE00000080140026843681143016003B11847C0
:102AF00070470000024AD36843F0C003D3607047B8
:102B000000380140024AD36843F0C003D3607047E5
:102B1000004400402DE9F041D0F89C600546F7687C
:102B20003368DA059CB20DD5202383F311884FF466
:102B300000710430FFF7D6FF6FF480733360002319
:102B400083F31188202383F3118805F1040814F01E
:102B50002F0333D183F31188380615D5210613D5F9
:102B6000202383F3118805F1380000F039FA00289A
:102B700046DA0821281DFFF7B5FF4FF67F733B406B
:102B8000F360002383F311887A060ED563060CD513
:102B9000202383F31188EA6C2B6D9A4202D12B6CAF
:102BA000002B2FD1002383F31188D5F8A420D368FC
:102BB000002B31D0BDE8F04110691847230713D02E
:102BC00014F0080F0CBF00218021E00748BF41F03E
:102BD0002001A20748BF41F04001630748BF41F40C
:102BE00080714046FFF77EFFA406736805D595F80F
:102BF000A0102846194000F093FA3468A4B2A6E762
:102C00007060BEE727F040073F041021281D3F0CED
:102C1000FFF768FFF760C5E7BDE8F08108B5034836
:102C2000FFF778FFBDE8084000F0ACBD902300201E
:102C300008B50348FFF76EFFBDE8084000F0A2BDED
:102C40003824002010B5094C094A2046002100F024
:102C500047FA084B084AC4F89C30084C002120462B
:102C600000F03EFA064BC4F89C3010BD90230020C3
:102C7000F52A000800380140052B00083824002000
:102C80000044004000F16043090103F56143C9B20B
:102C900083F80013012300F01F024009800000F1B7
:102CA0006040934000F56140C0F880310360704798
:102CB000090100F16040C9B200F56D40017670472E
:102CC000FFF7BCBD01230370002300F108028260FE
:102CD000C26000F1100283614360436202610363DA
:102CE0004261C363C36103628362C36243638363FC
:102CF000036443648364C3640365704710B5202391
:102D0000044683F31188022341600370FFF7BAFD84
:102D100003232370002383F3118810BD2DE9F041B4
:102D20001F4604460D461646202383F3118800F102
:102D300008082378042B0ED029462046FFF7C8FD4B
:102D400048B1204632462946FFF7E2FD002080F3D5
:102D50001188BDE8F0813946404600F0FDFA0028B0
:102D6000E7D0002383F31188BDE8F0812DE9F0411D
:102D70001F4604460D461646202383F3118800F1B2
:102D800010082378042B0ED029462046FFF7F8FDC3
:102D900048B1204632462946FFF70AFE002080F35C
:102DA0001188BDE8F0813946404600F0D5FA002888
:102DB000E7D0002383F31188BDE8F081F8B515460C
:102DC00082680B46AA428169066938BF8568761A0F
:102DD000B542044607D218462A46FEF797FBA36978
:102DE0002B44A3610DE011D932461846FEF78EFB45
:102DF000AF1B3A46E1683044FEF788FBE2683A448C
:102E0000A261A36828465B1BA360F8BD18462A464A
:102E1000FEF77CFBE368E4E72DE9F0410446154644
:102E200083682669934238BF856840690F46361A21
:102E3000B54206D22A46FEF769FB63692B446361FB
:102E40000DE012D93246A5EB0608FEF75FFB4246BD
:102E5000B919E068FEF75AFBE26842446261A36870
:102E600028465B1BA360BDE8F0812A46FEF74EFBB7
:102E7000E368E4E710B50024C361029B0A440060E4
:102E800040608460C160816141610261036210BD84
:102E900008B582694369934201D1826882B9826828
:102EA000013282605A1C42611970426903699A4278
:102EB00001D3C3684361002100F05EFA002008BD21
:102EC0004FF0FF3008BD000070B5202304460E46C9
:102ED00083F31188A568A5B1A368A269013BA3602B
:102EE000531CA36115782269934224BFE368A36150
:102EF000E3690BB120469847002383F311882846E5
:102F000070BD3146204600F027FA0028E2DA85F34A
:102F1000118870BD2DE9F74F05460F4690469A4639
:102F2000D0F81C90202686F311884FF0000B144631
:102F300064B1224639462846FFF740FF034668B988
:102F40005146284600F008FA0028F1D0002383F308
:102F50001188A8EB040003B0BDE8F08FB9F1000FB1
:102F600003D001902846C847019B8BF31188E41ACF
:102F70001F4486F31188DBE7C361009BC160816158
:102F800041611144006040608260016103627047EA
:102F9000F8B504460E461746202383F31188A5682A
:102FA000A5B1A368013BA36063695A1C62611E70EE
:102FB000236962699A4224BFE3686361E3690BB1E4
:102FC00020469847002080F31188F8BD39462046F6
:102FD00000F0C2F90028E2DA85F31188F8BD00009C
:102FE0008369426910B59A4201D182687AB98268D0
:102FF000013282605A1C82611C7803699A4201D3B3
:10300000C3688361002100F0B7F9204610BD4FF07E
:10301000FF3010BD2DE9F74F05460F4690469A4602
:10302000D0F81C90202686F311884FF0000B144630
:1030300064B1224639462846FFF7EEFE034668B9DA
:103040005146284600F088F90028F1D0002383F388
:103050001188A8EB040003B0BDE8F08FB9F1000FB0
:1030600003D001902846C847019B8BF31188E41ACE
:103070001F4486F31188DBE702684368114301604F
:1030800003B11847704700001430FFF743BF00003A
:103090004FF0FF331430FFF73DBF00003830FFF72B
:1030A000B9BF00004FF0FF333830FFF7B3BF000067
:1030B0001430FFF709BF00004FF0FF311430FFF765
:1030C00003BF00003830FFF763BF00004FF0FF324E
:1030D0003830FFF75DBF000000207047FFF7B2BD3A
:1030E0000E4B37B50360002343608360C360012348
:1030F000044615460374202200900B4600F15C0143
:103100001430FFF7B7FE00942B46202204F17C0117
:1031100004F13800FFF730FF03B030BD6846000807
:1031200038B5C36904460D461BB904210844FFF7AE
:10313000A3FF294604F11400FFF7AAFE002806DACF
:10314000201D4FF48061BDE83840FFF795BF38BDC2
:103150000022024B1B605B609A607047E0240020F5
:10316000002382680374054B1B6899689142FBD267
:103170005A6803604260106058607047E024002085
:1031800008B5202383F31188037C032B05D0042B7F
:103190000DD02BB983F3118808BD002243691A6052
:1031A0004FF0FF334361FFF7DBFF0023F2E790E8C6
:1031B0000C001A6002685360F2E700000023826886
:1031C0000374054B1B6899689142FBD85A680360E9
:1031D0004260106058607047E0240020054B196978
:1031E00008741868026853601A6018610123037438
:1031F000FDF7BCBAE024002030B54B1C87B0054673
:103200000A4C10D023690A4A01A800F0DDF82846CC
:10321000FFF7E4FF049B13B101A800F0EFF8236966
:10322000586907B030BDFFF7D9FFF8E7E024002068
:103230008131000838B50C4D41612B6981689A686D
:103240000446914203D8BDE83840FFF789BF1846CD
:10325000FFF786FF01232C61014623742046BDE859
:103260003840FDF783BA00BFE0240020044B1A6801
:103270001B6990689B68984294BF002001207047AA
:10328000E024002010B5084C236820691A685460B7
:103290002260012223611A74FFF790FF0146206922
:1032A000BDE81040FDF762BAE024002008B5FFF742
:1032B000DDFF18B1BDE80840FFF7E4BF08BD00001E
:1032C0008260022202740022427470478368A3F174
:1032D0003C0243F80C2C026943F83C2C426943F849
:1032E000382C074A43F81C2CC268A3F1180043F895
:1032F000102C022203F8082C002203F8072C704738
:103300007D07000810B5202383F31188FFF7DEFF47
:1033100000210446FFF78EFF002383F31188204627
:1033200010BD0000024B1B6958610F20FFF756BF0C
:10333000E0240020202383F31188FFF7F3BF00006F
:1033400008B50146202383F311880820FFF754FFB6
:10335000002383F3118808BD49B1064B42681B69FD
:1033600018605A60136043600420FFF745BF4FF0B8
:10337000FF307047E02400200368984206D01A68A6
:103380000260506059611846FFF7EABE70470000BE
:1033900038B504460D462068844200D138BD036824
:1033A00023605C604561FFF7DBFEF4E7054B03F14A
:1033B00014025A619A614FF0FF32DA6100221A62F8
:1033C000704700BFE024002010B5C2600A4A0361C4
:1033D00053699C68A1420CD85C680360446020601B
:1033E000586081609868411A99604FF0FF33D3614B
:1033F00010BD091B1B68ECE7E0240020036881680E
:103400009A680A449A604268136003685A6000230D
:103410004FF0FF32C360014BDA617047E0240020B7
:1034200000207047FEE70000704700004FF0FF30BB
:1034300070470000BFF34F8F024AD368DB07FCD40C
:10344000704700BF0020024008B5074B1B7853B9F6
:10345000FFF7F0FF054B1A69120641BF044A5A6094
:1034600002F188325A6008BD302500200020024059
:103470002301674508B5054B1B7833B9FFF7DAFF21
:10348000034A136943F08003136108BD302500200F
:10349000002002407F289ABF00F500308002002003
:1034A000704700004FF48060704700008020704734
:1034B0007F2808B50BD8FFF7EDFF00F580630268A1
:1034C000013204D104308342F9D1012008BD00202B
:1034D00008BD00007F2810B504461CD8FFF7AAFFDE
:1034E000FFF7B2FFF3220D4BDA6002221A61FFF7F9
:1034F000D1FF58611A6942F040021A61FFF79AFF42
:103500004FF4806100F004F9FFF7B4FF2046BDE8F6
:103510001040FFF7CDBF002010BD00BF00200240CB
:103520002DE9F84312F00103144606D040F236228A
:103530001F4B1A600020BDE8F88385181D4A95428C
:1035400004D940F23B211A4A1160F3E7FFF77CFFF0
:10355000FFF770FF4FF00109DFF86880451A012C72
:1035600005EB01060F4604D8FFF784FF0120BDE8F4
:10357000F883C8F8109031F8023B3380FFF75AFF08
:103580000020C8F8100033883A889BB29A420DD0C8
:1035900040F25222064B1A60074B1E60074B1C601C
:1035A000074B1F60FFF766FFBDE8F883023CD6E7D4
:1035B0002C250020FFFF01082025002028250020C1
:1035C0002425002000200240084908B50B7828B1C6
:1035D00053B9FFF739FF01230B7008BD23B1BDE8D4
:1035E00008400870FFF746BF08BD00BF3025002027
:1035F0004FF47A700D4B30B51B6A58430C4B1A6868
:1036000090421A460FD20B4B0B49D3E9004514F1F7
:10361000FF3445F10005C3E900450B6803F583035A
:1036200003F637130B60106030BD00BFE0240020AC
:1036300034250020402500203825002070B500F0FA
:1036400047F90646FFF7D4FF054BD3E90045241898
:1036500045F10005304600F045F92046294670BD89
:103660004025002038B500F033F94FF47A74054650
:10367000FFF7BEFFB0FBF4F4034B18680444284680
:1036800000F030F9204638BD3825002010B5094C2F
:103690000439013AD2B2FF2A00D110BD5308980074
:1036A000043054F8233000599BB243EA004341F8F8
:1036B000043FEEE7046C004030B50748013AD2B24F
:1036C000FF2A00D130BD0D88540840F82450A300D3
:1036D0004C8804331C50F1E7046C004007B501220C
:1036E00001A90020FFF7D2FF019803B05DF804FBA9
:1036F00013B50446FFF7F2FFA04206D002A941F835
:10370000044D01220020FFF7D7FF02B010BD0000DA
:103710007047000045F25552064B1A6002225A606B
:1037200040F6FF729A604CF6CC421A600122024BBE
:103730001A7070470030004049250020034B1B6879
:103740009B0042BF0122024B1A70704724100240B6
:10375000482500204FF08072014B1A60704700BF6F
:1037600024100240014B1878704700BF4825002004
:10377000EFF30983203383F30988002383F311884F
:103780007047000010B5202383F311880D4B5B6850
:1037900013F4006312D0EFF309844FF0807344F800
:1037A000043CA4F1200383F30988FFF75FFD18B1FF
:1037B000054B44F8083C10BD044BFAE783F311882D
:1037C00010BD00BF00ED00E08D0700089007000865
:1037D00070470000FEE70000084A094B09498B4288
:1037E00004D30021084A934205D3704752F8040FCE
:1037F00043F8040BF3E743F8041BF4E7A44700087D
:10380000042600200426002004260020FEE70000F5
:1038100010B5174CFFF79CFCFFF7C8FD8022154937
:103820002046FFF74DFD012344F8180C0374124B9A
:10383000124AD96821F4E0610904090C0A431049CD
:10384000DA60CA6842F08072CA600E490A6842F0C3
:1038500001020A601022DA77202283F82220002356
:1038600083F3118862B6BDE810400748FFF74ABDF0
:10387000082500209046000800ED00E00003FA054E
:10388000F0ED00E0001000E098460008F8B50F4C9D
:10389000226A01322262224652F8141F91421546D2
:1038A00006D020268B68013B8B6063699A6802B161
:1038B000F8BD1968DF68DA604D60616182F31188D4
:1038C0001869B84786F31188EFE700BFE0240020AD
:1038D000EFF3118020B9EFF30583202282F31188E2
:1038E0007047000010B558B9EFF30584C4F308041D
:1038F00014B180F3118810BDFFF7D8FC84F3118850
:1039000010BD000000F030B808B500F063F9FFF713
:103910007FFFBDE80840FFF711BF000070470000BF
:103920004FF0FF310E4B1A6919611A6900221A61B2
:103930001869D868D960D968DA60DA68DA6942F05B
:103940008052DA61DA69DA6942F00062DA61054AC6
:10395000DB69136843F48073136000F01BB900BF88
:103960000010024000700040194B1A6842F001023A
:103970001A601A689007FCD51A6802F0F9021A60FA
:1039800000225A605A6812F00C0FFBD11A6842F4F8
:1039900080321A601A689103FCD55A6842F4E81222
:1039A0005A601A6842F080721A601A689201FCD557
:1039B0001221084A5A60084A11605A6842F002020D
:1039C0005A605A6802F00C02082AFAD1704700BF08
:1039D0000010024000641D0000200240084A08B5A3
:1039E000536911680B4003F00103536123B1054A89
:1039F00013680BB150689847BDE80840FFF7C2BE96
:103A00000004014010230020084A08B553691168DA
:103A10000B4003F00203536123B1054A93680BB1D5
:103A2000D0689847BDE80840FFF7ACBE00040140ED
:103A300010230020084A08B5536911680B4003F0B1
:103A40000403536123B1054A13690BB150699847C8
:103A5000BDE80840FFF796BE000401401023002097
:103A6000084A08B5536911680B4003F00803536115
:103A700023B1054A93690BB1D0699847BDE8084066
:103A8000FFF780BE0004014010230020084A08B55B
:103A9000536911680B4003F01003536123B1054AC9
:103AA000136A0BB1506A9847BDE80840FFF76ABE39
:103AB0000004014010230020174B10B55C691A6800
:103AC000144004F478725A61A30604D5134A936A29
:103AD0000BB1D06A9847600604D5104A136B0BB13E
:103AE000506B9847210604D50C4A936B0BB1D06BF1
:103AF0009847E20504D5094A136C0BB1506C9847FE
:103B0000A30504D5054A936C0BB1D06C9847BDE86A
:103B10001040FFF737BE00BF000401401023002013
:103B20001A4B10B55C691A68144004F47C425A615F
:103B3000620504D5164A136D0BB1506D98472305E5
:103B400004D5134A936D0BB1D06D9847E00404D5AA
:103B50000F4A136E0BB1506E9847A10404D50C4A5E
:103B6000936E0BB1D06E9847620404D5084A136F68
:103B70000BB1506F9847230404D5054A936F0BB1DE
:103B8000D06F9847BDE81040FFF7FCBD000401402E
:103B900010230020062108B50846FFF773F8062118
:103BA0000720FFF76FF806210820FFF76BF80621C2
:103BB0000920FFF767F806210A20FFF763F80621BE
:103BC0001720FFF75FF8BDE8084006212820FFF71F
:103BD00059B8000008B5FFF7A3FE0648FEF740FFFE
:103BE000FFF76EF8FFF77AFAFFF798FEBDE8084096
:103BF00000F002B8B846000800F00EB808B520235F
:103C000083F31188FFF742FE002383F31188BDE898
:103C10000840FFF7B7BD0000054B064A08215A606F
:103C200000229A6007220B201A60FFF741B800BFFC
:103C300010E000E03F1901001FB51C46094B054686
:103C40001B68D86852B1084B8DE80A0002922B46D7
:103C500022460649FDF778FC00F042F8044B1A466C
:103C6000F2E700BF14110020F446000801470008E5
:103C7000F33D000810B501390244904201D1002003
:103C800010BD10F8013B11F8014FA342F5D0181BED
:103C900010BD00002DE9F8430746884691461E46B0
:103CA0008BB10D46A8EB0500B54207EB000402D22C
:103CB0000020BDE8F883324649462046FFF7DAFF88
:103CC00018B1013DEEE7BDE8F8832046BDE8F88372
:103CD000034611F8012B03F8012B002AF9D1704794
:103CE00008B5062000F02CF80120FFF79BFB000030
:103CF0001F2938B504460D4604D9162303604FF03A
:103D0000FF3038BD426C12B152F821304BB9204619
:103D100000F030F82A4601462046BDE8384000F061
:103D200017B8012B0AD0591C03D1162303600120B8
:103D300038BD0024284642F825409847002038BD69
:103D4000024B01461868FFF7D3BF00BF14110020D3
:103D500038B50023064C0546084611462360FFF798
:103D600065FB431C02D1236803B12B6038BD00BF43
:103D700000260020FFF754BB40A2E4F164689106DE
:103D80004E6F20617070207369670A004261642081
:103D90006677206C656E6774682025750A0042613D
:103DA0006420626F6172645F6964202575207368A6
:103DB0006F756C642062652025750A00426164207D
:103DC00061707020435243203078253038783A3083
:103DD0007825303878203078253038783A30782592
:103DE0003038780A00476F6F64206669726D7761BA
:103DF00072650A0072656365697665645F756E69F0
:103E00007175655F69645F6C656E203C2055415635
:103E100043414E5F50524F544F434F4C5F44594EB5
:103E2000414D49435F4E4F44455F49445F414C4CCF
:103E30004F434154494F4E5F554E495155455F4997
:103E4000445F4D41585F4C454E475448002E2E2F3D
:103E50002E2E2F546F6F6C732F41505F426F6F7413
:103E60006C6F616465722F63616E2E6370700061A8
:103E70006C6C6F63617465645F6E6F64655F6964C9
:103E8000203C3D20313237006F72672E61726475BD
:103E900070696C6F742E61705F7065726970680014
:103EA000766F69642068616E646C655F616C6C6FCD
:103EB000636174696F6E5F726573706F6E7365288E
:103EC00043616E617264496E7374616E63652A2C1E
:103ED0002043616E61726452785472616E736665DC
:103EE000722A290000000000963007772C610EEE40
:103EF000BA51099919C46D078FF46A7035A563E941
:103F0000A395649E3288DB0EA4B8DC791EE9D5E067
:103F100088D9D2972B4CB609BD7CB17E072DB8E766
:103F2000911DBF906410B71DF220B06A4871B9F3BB
:103F3000DE41BE847DD4DA1AEBE4DD6D51B5D4F4F4
:103F4000C785D38356986C13C0A86B647AF962FD59
:103F5000ECC9658A4F5C0114D96C0663633D0FFAA6
:103F6000F50D088DC8206E3B5E10694CE44160D5AC
:103F7000727167A2D1E4033C47D4044BFD850DD296
:103F80006BB50AA5FAA8B5356C98B242D6C9BBDBA9
:103F900040F9BCACE36CD832755CDF45CF0DD6DCA4
:103FA000593DD1ABAC30D9263A00DE518051D7C84B
:103FB0001661D0BFB5F4B42123C4B3569995BACFD6
:103FC0000FA5BDB89EB802280888055FB2D90CC6F7
:103FD00024E90BB1877C6F2F114C6858AB1D61C170
:103FE0003D2D66B69041DC760671DB01BC20D2988F
:103FF0002A10D5EF8985B1711FB5B606A5E4BF9F1C
:1040000033D4B8E8A2C9077834F9000F8EA809960E
:1040100018980EE1BB0D6A7F2D3D6D08976C649179
:10402000015C63E6F4516B6B62616C1CD830658592
:104030004E0062F2ED95066C7BA5011BC1F408826F
:1040400057C40FF5C6D9B06550E9B712EAB8BE8BB0
:104050007C88B9FCDF1DDD62492DDA15F37CD38C39
:10406000654CD4FB5861B24DCE51B53A7400BCA337
:10407000E230BBD441A5DF4AD795D83D6DC4D1A469
:10408000FBF4D6D36AE96943FCD96E34468867AD40
:10409000D0B860DA732D0444E51D03335F4C0AAADF
:1040A000C97C0DDD3C710550AA41022710100BBEE2
:1040B00086200CC925B56857B3856F2009D466B929
:1040C0009FE461CE0EF9DE5E98C9D9292298D0B05E
:1040D000B4A8D7C7173DB359810DB42E3B5CBDB70B
:1040E000AD6CBAC02083B8EDB6B3BF9A0CE2B6038C
:1040F0009AD2B1743947D5EAAF77D29D1526DB0441
:104100008316DC73120B63E3843B64943E6A6D0D8B
:10411000A85A6A7A0BCF0EE49DFF099327AE000AD6
:10412000B19E077D44930FF0D2A3088768F2011E69
:10413000FEC206695D5762F7CB67658071366C1900
:10414000E7066B6E761BD4FEE02BD3895A7ADA1021
:10415000CC4ADD676FDFB9F9F9EFBE8E43BEB71702
:10416000D58EB060E8A3D6D67E93D1A1C4C2D8388C
:1041700052F2DF4FF167BBD16757BCA6DD06B53FF2
:104180004B36B248DA2B0DD84C1B0AAFF64A033631
:10419000607A0441C3EF60DF55DF67A8EF8E6E31B0
:1041A00079BE69468CB361CB1A8366BCA0D26F25F9
:1041B00036E2685295770CCC03470BBBB916022246
:1041C0002F260555BE3BBAC5280BBDB2925AB42B5B
:1041D000046AB35CA7FFD7C231CFD0B58B9ED92C70
:1041E0001DAEDE5BB0C2649B26F263EC9CA36A75D5
:1041F0000A936D02A906099C3F360EEB856707728C
:1042000013570005824ABF95147AB8E2AE2BB17BF2
:10421000381BB60C9B8ED2920DBED5E5B7EFDC7C79
:1042200021DFDB0BD4D2D38642E2D4F1F8B3DD68D0
:104230006E83DA1FCD16BE815B26B9F6E177B06FCB
:104240007747B718E65A0888706A0FFFCA3B0666B8
:104250005C0B0111FF9E658F69AE62F8D3FF6B6145
:1042600045CF6C1678E20AA0EED20DD75483044EE7
:10427000C2B30339612667A7F71660D04D47694975
:10428000DB776E3E4A6AD1AEDC5AD6D9660BDF4088
:10429000F03BD83753AEBCA9C59EBBDE7FCFB2473B
:1042A000E9FFB5301CF2BDBD8AC2BACA3093B35320
:1042B000A6A3B4240536D0BA9306D7CD2957DE5429
:1042C000BF67D9232E7A66B3B84A61C4021B685D02
:1042D000942B6F2A37BE0BB4A18E0CC31BDF055A7B
:1042E0008DEF022D63616E617264496E6974000026
:1042F00063616E6172645365744C6F63616C4E6F81
:10430000646549440000000063616E617264486145
:104310006E646C6552784672616D650063616E61B2
:1043200072644465636F64655363616C617200001D
:1043300063616E617264456E636F64655363616C43
:1043400061720000696E6372656D656E74547261AE
:104350006E73666572494400656E71756575655466
:10436000784672616D657300707573685478517525
:104370006575650070726570617265466F724E6535
:1043800078745472616E736665720000636F707941
:104390004269744172726179000000006465736360
:1043A00061747465725472616E736665725061797E
:1043B0006C6F61640000000066726565426C6F633B
:1043C0006B0000006269745F6C656E677468203E04
:1043D00020300072656D61696E696E675F62697435
:1043E00073203E203000696E7075745F6269745F7F
:1043F0006F6666736574203E3D20626C6F636B5F11
:104400006269745F6F666673657400626C6F636B7C
:104410005F656E645F6269745F6F66667365742062
:104420003E20626C6F636B5F6269745F6F66667378
:1044300065740072656D61696E696E675F6269744B
:104440005F6C656E677468203C3D2072656D6169C4
:104450006E696E675F6269747300696E7075745F10
:104460006269745F6F6666736574203C3D20747288
:10447000616E736665722D3E7061796C6F61645F09
:104480006C656E202A2038006F75747075745F62D9
:1044900069745F6F6666736574203C3D2036340036
:1044A00072656D61696E696E675F6269745F6C6584
:1044B0006E677468203D3D20300028726573756C0E
:1044C00074203E2030292026262028726573756CC2
:1044D00074203C3D2036342920262620287265731E
:1044E000756C74203C3D206269745F6C656E677406
:1044F0006829000064657374696E6174696F6E2069
:10450000213D202828766F6964202A2930290076E9
:10451000616C756520213D202828766F6964202A0A
:10452000293029006F66667365745F7769746869FE
:104530006E5F626C6F636B203C2028333255202DF8
:10454000205F5F6275696C74696E5F6F6666736524
:10455000746F66202843616E617264427566666599
:1045600072426C6F636B2C206461746129290000B6
:104570006F75745F696E7320213D202828766F69FE
:1045800064202A29302900007372635F6C656E20F5
:104590003E203055000000002863616E5F69642092
:1045A0002620307831464646464646465529203D27
:1045B0003D2063616E5F696400000000616C6C6F98
:1045C0006361746F722D3E7374617469737469638F
:1045D000732E63757272656E745F75736167655F64
:1045E000626C6F636B73203E203000007472616EEA
:1045F000736665725F696420213D202828766F69A3
:1046000064202A293029000073746174652D3E628C
:1046100075666665725F626C6F636B73203D3D20EB
:104620002828766F6964202A293029002E2E2F2E03
:104630002E2F6D6F64756C65732F6C696263616E8C
:104640006172642F63616E6172642E6300697465C8
:104650006D2D3E6672616D652E646174615F6C657F
:104660006E203E203000000000000000A530000851
:1046700091300008CD300008B9300008C53000087E
:10468000B13000089D30000889300008D93000089A
:104690006D61696E00000000B046000850250020E2
:1046A00000260020010000000D3800080000000076
:1046B00069646C65000000000C1E0000887B818826
:1046C000B85789880000000088888884888888888E
:1046D000000000008888888888888888000000009A
:1046E000888888888888888800000000888888886A
:1046F000888888882C2066756E6374696F6E3A208E
:1047000000617373657274696F6E202225732220B5
:104710006661696C65643A2066696C652022257360
:10472000222C206C696E65202564257325730A0090
:10473000FFFFFFFF6400000000000000FE2A0100F0
:10474000D20400001811002000000000000000004A
:104750000000000000000000000000000000000059
:104760000000000000000000000000000000000049
:104770000000000000000000000000000000000039
:104780000000000000000000000000000000000029
:104790000000000000000000000000000000000019
:0847A000000000000000000011
:00000001FF
